:060000000CEF00F001000E
:0E0006001200D8CFFFF5FACFFEF52BEF1AF05F
:10001800100EE96E000EEA6E5D0EE16E020EE26EE3
:10002800F8EC02F0AB0EE96E050EEA6EE20EE16E38
:10003800050EE26EF8EC02F0E80EE96E000EEA6ECC
:10004800000EE16E010EE26E840EF66E000EF76E83
:10005800000EF86E89EC2DF0AA0EE96E050EEA6E18
:10006800AB0EE16E050EE26E040EF66E000EF76E34
:10007800000EF86E89EC2DF07FEF1AF02707E006E6
:100088004E0700073811211105114A11BB119A11A9
:100098006211E8102A0096D000012E0E596F000E4A
:1000A8005A6F00011C0E5B6F5C6BACEC23F0C6EC66
:1000B80023F000012E0E4A6F000E4B6F62D900012B
:1000C8002E51010A2F11D8B401D006D032C0E8FF52
:1000D800060AD8B402D000D007D000D033C0E8FF59
:1000E800040AD8B402D000D002D000D002D0000E4A
:1000F80068D02CC0E1FF2DC0E2FF2AC0D9FF2BC079
:10010800DAFF00013451020A3511D8A401D001D018
:1001180003D0000EE76E0FD000013451010A3511EB
:10012800D8A401D001D003D0010EE76E04D0020E8E
:10013800E76E000E46D032C2E8FF000146630AD0DF
:1001480000D0330EE96E020EEA6EEF50476302D01C
:1001580000D001D009D0340EE96E020EEA6EEF50DD
:10016800486302D000D001D009D0350EE96E020EE6
:10017800EA6EEF50496302D000D002D000D01FD001
:10018800360E006E000E016E00C0E9FF01C0EAFFE6
:10019800D9CFE1FFDACFE2FF060E90EC2DF0060E84
:1001A800D924E96E000EDA20EA6E3CC0EEFF3DC0AD
:1001B800EEFF3EC0EEFF3FC0EEFF010E02D0000E84
:1001C80000D0120069D72A00DAD02AC0D9FF2BC084
:1001D800DAFF0001010E2D6F2E6B0001000E2F6F4C
:1001E800080E306F060EE8CF31F0040EE8CF32F07B
:1001F80000012C05D8A401D001D017D00001010EB0
:10020800336F346BFF0EE8CF3FF0FF0EE8CF40F0BE
:10021800FF0EE8CF41F0FF0EE8CF42F0FF0EE8CF27
:1002280043F0FF0EE8CF44F013D00001020E336F05
:10023800346BD9CF00F0DACF01F000C0E9FF01C07C
:10024800EAFF3F0EE16E000EE26E060E90EC2DF016
:1002580036C235F037C236F038C237F039C238F016
:100268003AC239F03BC23AF032C23BF033C23CF0FA
:1002780034C23DF035C23EF03CC200F0060ED9242F
:10028800E96E000EDA20EA6EEF50016E00010150AF
:100298003B190014D8B401D010D03DC200F0070EAD
:1002A800D924E96E000EDA20EA6EEF50016E015093
:1002B8003C190014D8B402D000D011D000D03EC2EE
:1002C80000F0080ED924E96E000EDA20EA6EEF502D
:1002D800016E01503D190014D8B402D000D011D0DD
:1002E80000D03FC200F0090ED924E96E000EDA20D2
:1002F800EA6EEF50016E01503E190014D8B402D0D6
:1003080000D002D000D009D040C245F041C246F02A
:1003180042C247F043C248F010D0060ED924E96E15
:10032800000EDA20EA6EEECF45F0EECF46F0EECFC3
:1003380047F0EDCF48F0ED52ED5200012D0E4A6F17
:10034800000E4B6F1ED800013F0EDA6F000EDB6FF8
:10035800060EE8CFDCF000011C0EDD6FDE6BE2EC70
:1003680023F000012D0EDA6F000EDB6F00011C0E6A
:10037800DC6FDD6B13EC24F02FEC24F0120025D792
:100388004A004ED04AC0E9FF4BC0EAFFEECF00F06A
:10039800EDCF01F000C0DCF001C0DDF021EC26F06B
:1003A8004AC0E9FF4BC0EAFF00C0EEFF01C0EDFF05
:1003B8000001020E4A25E96E000E4B21EA6EEECFCF
:1003C80000F0EDCF01F000C0DCF001C0DDF021EC61
:1003D80026F00001020E4A25E96E000E4B21EA6E56
:1003E80000C0EEFF01C0EDFF060E4A25E96E000EC3
:0803F8004B21EA6EEECF00F08C
:10040000EDCF01F000C0DCF001C0DDF021EC26F002
:100410000001060E4A25E96E000E4B21EA6E00C06F
:10042000EEFF01C0EDFF1200B1D73D0003D0000187
:100430003D4B3E2B3DC0F6FF3EC0F7FF050EF76477
:1004400003D00800F55005D0F6CFE9FFF7CFEAFF5B
:10045000EF50200AD8B4EBD73DC0F6FF3EC0F7FFFF
:10046000050EF76403D00800F55005D0F6CFE9FF7C
:10047000F7CFEAFFEF50090A0001D8B4D9D7406B93
:10048000416B3F6B3DC0F6FF3EC0F7FF050EF764C2
:1004900003D00800F55005D0F6CFE9FFF7CFEAFF0B
:1004A000EF502D0AD8A402D03F2B13D03DC0F6FF49
:1004B0003EC0F7FF050EF76403D00800F55005D0E5
:1004C000F6CFE9FFF7CFEAFFEF502B0AD8A403D00D
:1004D00000013D4B3E2B3DC0F6FF3EC0F7FF050E31
:1004E000F76403D00800F55005D0F6CFE9FFF7CF49
:1004F000EAFFEF5079EC2DF0D8A025D00A0E026E5D
:10050000036A40C000F041C001F06BEC2DF03DC02B
:10051000F6FF3EC0F7FF050EF76403D00800F55064
:1005200005D0F6CFE9FFF7CFEAFFEF500424006EC5
:10053000000E0520016ED00E00240001406FFF0E5A
:100540000120416FC6D700013F5140C000F041C0BB
:1005500001F0D8B41200001E011E002AD8B4012AEE
:10056000120003D00501AB6B1200FCD73FD036D090
:100570000001200E2A6F000E2B6F00011F0E2C6F42
:10058000000E2D6F4FEC00F0006E016A015000105C
:10059000D8A401D001D001D026D000011F510009FC
:1005A000D8A401D001D001D01ED0010EE8CFABF508
:1005B00036EC23F00009D8B401D001D00CD00001F2
:1005C000200E2A6F000E2B6F00012C6BE8EC00F060
:1005D0000501AB6B02D0000E08D005D0ABC5E8FF1B
:1005E000000AC6E0E5D7010E00D01200C0D7EE6ABF
:0E05F000EA50E262FCD7E950E162F9D712004E
:100600005458540048544D00474946004347490058
:100610004A504700434C4100574156007465787476
:100620002F706C61696E0000000000000000000087
:10063000746578742F68746D6C0000000000000011
:1006400000000000696D6167652F67696600000042
:100650000000000000000000746578742F68746D5D
:100660006C0000000000000000000000696D616780
:10067000652F6A7065670000000000000000000040
:100680006170706C69636174696F6E2F6A61766105
:100690002D766D00617564696F2F782D77617665B1
:1006A0000000000000000000485454502F312E304C
:1006B00020323030204F4B0D0A436F6E74656E74DC
:1006C0002D747970653A20000D0A0D0A00474554D3
:1006D00000504F535400494E4445582E48544D0045
:1006E000485454502F312E3020323030204F4B0D93
:1006F0000A436F6E74656E742D747970653A2000CC
:10070000485454502F312E3020353033200D0A0DEF
:100710000A5365727669636520556E617661696C0E
:1007200061626C650D0A00485454502F312E302000
:10073000343034204E6F7420666F756E640D0A0D70
:100740000A4E6F7420666F756E642E0D0A000D0AD6
:100750000D0A003C68746D6C3E3C686561643E3C0B
:100760007469746C653E5765622053657276657274
:1007700020492F4F20436F6E74726F6C3C2F746949
:10078000746C653E3C2F686561643E3C626F6479C1
:100790003E3C63656E7465723E3C666F6E742066A7
:1007A0006163653D68656C7665746963613E3C684C
:1007B000323E3C753E4F757470757420436F6E7495
:1007C000726F6C3C2F753E3C2F68323E3C464F5258
:1007D0004D204D4554484F443D4745542061637476
:1007E000696F6E3D303E3C7461626C6520626F7271
:1007F0006465723D323E3C74723E3C74643E3C69BA
:100800006E70757420747970653D7375626D69746E
:10081000206E616D653D312076616C75653D4436B5
:100820003D2530313E3C2F74643E3C74643E3C694F
:100830006E70757420747970653D7375626D69743E
:10084000206E616D653D302076616C75653D443587
:100850003D2530303E3C2F74643E3C2F74723E3C4C
:100860002F7461626C653E3C2F666F726D3E3C2F4B
:10087000626F64793E3C2F68746D6C3E04FFFFFF2D
:100880003C48544D4C3E3C484541443E3C54495400
:100890004C453E4D6963726F6368697020544350E4
:1008A0002F495020537461636B2044656D6F3C2F5A
:1008B0005449544C453E3C2F484541443E3C4652E9
:1008C000414D4553455420726F77733D223130308E
:1008D0002C33302220626F726465723D303E2020DE
:1008E0003C4652414D45206E616D653D22746F70EE
:1008F0002220097372633D226D61696E2E68746DEA
:1009000022206D617267696E6865696768743D353C
:10091000206D617267696E77696474683D353E0960
:100920003C4652414D4553455420636F6C733D2204
:1009300038302C38302220626F726465723D303E50
:10094000202009093C4652414D45206E616D653DB0
:10095000226C656674222020207372633D225374DA
:10096000617475732E63676922206D617267696EA9
:100970006865696768743D32206D617267696E777A
:10098000696474683D323E202009093C4652414D5D
:1009900045206E616D653D22726967687422202072
:1009A000207372633D22436F6D6D616E64732E63BD
:1009B000676922206D617267696E6865696768742E
:1009C0003D32206D617267696E77696474683D328B
:1009D0003E093C2F4652414D455345543E3C2F461F
:1009E00052414D455345543E3C2F48544D4C3E04D6
:1009F000FFFFFF3C48544D4C3E3C484541443E3C83
:100A00002F484541443E3C424F44593E3C666F6E40
:100A10007420666163653D68656C766574696361C1
:100A20003E3C63656E7465723E3C423E3C553E3CC6
:100A3000464F4E542053495A453D3720434F4C4F63
:100A4000523D2223303030306666223E3C503E4DCF
:100A50006963726F63686970205443502F49502056
:100A6000537461636B3C2F503E3C2F423E3C2F55EC
:100A70003E3C2F464F4E543E3C2F63656E7465726C
:100A80003E5468697320697320612073616D706CD6
:100A900065207061676520696E74656E64656420A9
:100AA000746F2064656D6F6E737472617465204D30
:100AB0006963726F63686970205443502F495020F6
:100AC000537461636B206361706162696C697469FE
:100AD00065732E546869732070616765206973209F
:100AE00073657276656420627920485454502053AF
:100AF00065727665722C2072756E6E696E67206FF6
:100B00006E204D6963726F6368697020504943318C
:100B100038206D6963726F636F6E74726F6C6C6591
:100B2000722C7574696C697A696E67204D6963729D
:100B30006F63686970205443502F4950205374618B
:100B4000636B2E3C703E4D6963726F636869702001
:100B5000537461636B206F666665727320666F6C99
:100B60006C6F77696E672066656174757265733A3C
:100B70003C2F703E3C756C3E3C6C693E506F72740D
:100B800061626C65206163726F7373204D6963727B
:100B90006F636869702050494331382066616D6920
:100BA0006C79206F66206D6963726F636F6E74720B
:100BB0006F6C6C6572733C2F6C693E3C6C693E4394
:100BC0006F6F7065726174697665206D756C74699C
:100BD0007461736B696E67205443502F49502073C2
:100BE0007461636B3C2F6C693E3C6C693E55736568
:100BF0002069742061732070617274206F662048D0
:100C000054545020536572766572206F722063755C
:100C100073746F6D205443502F4950206261736587
:100C200064206170706C69636174696F6E3C2F6CD5
:100C3000693E3C6C693E4D756C7469706C652054FE
:100C4000435020736F636B657420737570706F729F
:100C5000743C2F6C693E3C6C693E485454502053A0
:100C600065727665722077697468206D756C746939
:100C7000706C6520636F6E6E656374696F6E732050
:100C8000737570706F72743C2F6C693E3C6C693E7A
:100C90005061676573206D61792062652073746FA0
:100CA00072656420696E20696E7465726E616C2075
:100CB00070726F6772616D206D656D6F7279206FF4
:100CC000722065787465726E616C20646174612055
:100CD000454550524F4D3C2F6C693E3C6C693E532C
:100CE0007570706F727420666F722048544D4C207E
:100CF000666F726D733C2F6C693E3C6C693E50436D
:100D00002062617365642070726F6772616D207418
:100D10006F20636F6E7665727420776562207061F4
:100D200067657320696E746F204D6963726F6368C5
:100D300069702046696C652053797374656D20284D
:100D40004D504653293C2F6C693E3C6C693E4D6FBB
:100D500064756C61722064657369676E20746F20BE
:100D6000656173696C7920616464206E65772063C6
:100D70006F6D706F6E656E74733C2F6C693E3C2FA7
:100D8000756C3E3C2F424F44593E3C2F48544D4CCD
:100D90003E04FFFFFF3C68746D6C3E3C6D65746102
:100DA00020687474702D65717569763D2272656670
:100DB000726573682220636F6E74656E743D2233B2
:100DC000223E3C686561643E3C7469746C653E57C4
:100DD0006562205365727665722053746174757311
:100DE0003C2F7469746C653E3C2F686561643E3CC1
:100DF000626F64793E3C63656E7465723E3C666FFB
:100E00006E7420666163653D68656C7665746963C0
:100E1000613E3C753E3C68323E53797374656D208B
:100E20005374617475733C2F68323E3C2F753E3CA1
:100E30007461626C6520626F726465723D323E3C23
:100E400074723E3C74643E53333D2530343C2F7401
:100E5000643E3C74643E44363D2530313C2F74641E
:100E60003E3C74643E44353D2530303C2F74643E36
:100E70003C74643E414E303D2530323C2F74643E1C
:100E80003C74643E414E313D2530333C2F74643E0A
:100E90003C2F74723E3C2F7461626C653E3C627202
:100EA0003E3C2F626F64793E3C2F68746D6C3E044B
:100EB000FFFFFF005307434F4D4D414E44532E4318
:100EC0004749008008494E4445582E48544D20203B
:100ED0002000F3094D41494E2E48544D202020203A
:100EE00000950D5354415455532E43474920200437
:100EF000FFFF454E44204F462046415420204D439D
:100F00004850537461636B2076322E3000426F611B
:100F100072642053657475702E2E2E0020202020C0
:100F200020202020202020202020202000434F4D62
:100F30004D414E44532E43474900494E4445582E97
:100F400048544D000D0A0D0A0D4D4348505374612D
:100F5000636B2044656D6F204170706C69636174D0
:100F6000696F6E2076312E3020284D6963726F6371
:100F7000686970205443502F495020537461636B4B
:100F800020322E30290D0A0D0A09313A20436861BA
:100F90006E676520426F6172642073657269616C6F
:100FA000206E756D6265722E0D0A09323A20436813
:100FB000616E67652064656661756C7420495020B8
:100FC000616464726573732E0D0A09333A204368B5
:100FD000616E67652064656661756C742067617415
:100FE0006577617920616464726573732E0D0A09F7
:100FF000343A204368616E67652064656661756C8C
:1010000074207375626E6574206D61736B2E0D0AAA
:1010100009353A20456E61626C6520444843502092
:101020002620495020476C65616E696E672E0D0A57
:1010300009363A2044697361626C65204448435024
:10104000202620495020476C65616E696E672E0D21
:101050000A09373A20446F776E6C6F6164204D50F7
:10106000465320696D6167652E0D0A09383A205391
:10107000617665202620517569742E0D0A0D0A458A
:101080006E7465722061206D656E752063686F698E
:1010900063652028312D38293A20000D0A496E76E3
:1010A000616C696420696E7075742072656365692E
:1010B000766564202D20496E7075742069676E6FA7
:1010C0007265642E0D0A507265737320616E79200B
:1010D0006B657920746F20636F6E74696E75652E11
:1010E0002E2E0D0A002575000D0A4E6F77207275A1
:1010F0006E6E696E67206170706C69636174696F90
:101100006E2E2E2E000D0A44656661756C742047A4
:101110006174657761792041646472657373202816
:10112000000D0A44656661756C7420495020416465
:1011300064726573732028000D0A53657269616CCF
:10114000204E756D6265722028000D0A4465666147
:10115000756C74205375626E6574204D61736B20DD
:1011600028000D0A526561647920746F20646F77DE
:101170006E6C6F6164204D50465320696D616765E8
:10118000202D2055736520586D6F64656D20707239
:101190006F746F636F6C2E0D0A000D0A4448435044
:1011A000202620495020476C65616E696E67206477
:1011B000697361626C65642E0D0A000D0A44484330
:1011C00050202620495020476C65616E696E67206B
:0C11D000656E61626C65642E0D0A000003
:1011DC00D96AD950220D100EF324E16E010EF420C1
:1011EC00E26EE76A210EE124E96E000EE220EA6E5F
:1011FC00EF50FE0BEF6E210EE124E96E000EE220A3
:10120C00EA6EEF50FD0B0209EF6E210EE124E96E40
:10121C00000EE220EA6EEF50FB0B0409EF6E210E7C
:10122C00E124E96E000EE220EA6EEF50EF0BEF6E58
:10123C00210EE124E96E000EE220EA6EEF50F70B6E
:10124C00EF6E0F0EE124E96E000EE220EA6EFF0E47
:10125C00EF6E1F0EE124E96E000EE220EA6E580ECE
:10126C00EE6E020EED6ED92A070ED95CD8A0B1D75E
:10127C000101006B040E016F0101046B056B066B21
:10128C00076B12001A00D96AD950220D100EF324E4
:10129C00E16E010EF420E26EE750D8A447D0010EA7
:1012AC00E76E0B0EE124E96E000EE220EA6E1AC026
:1012BC00EEFF1BC0EDFF0D0EE124E96E000EE220E7
:1012CC00EA6EEE6AED6A070EE124E96E000EE2208A
:1012DC00EA6EEE6AEE6AEE6AED6AED52ED52210E9E
:1012EC00E124E96E000EE220EA6EEF50FE0B0109DC
:1012FC00EF6E210EE124E96E000EE220EA6EEF5053
:10130C00F70BEF6E0F0EE124E96E000EE220EA6E91
:10131C00FF0EEF6E210EE124E96E000EE220EA6E64
:10132C00EF50FD0B0209EF6ED9501200D92A070EAF
:10133C00D95CD8B0FE0CA8D7D96E220D100EF324B0
:10134C00E96E010EF420EA6EEF50040A000ED8B4D8
:10135C00010E1200D96E220D100EF324E16E010E57
:10136C00F420E26ED95000017F6FE1CF80F0E2CF24
:10137C0081F0E750040AD8B406D080C082F081C056
:10138C0083F0ACEF10F000017F51FFD980C0E1FF7A
:10139C0081C0E2FF010EE124E8CF89F0000EE220CB
:1013AC00E8CF8AF00B0EE124E96E000EE220EA6E23
:1013BC00EECF00F0EDCF01F000C08BF001C08CF04F
:1013CC000D0EE124E96E000EE220EA6EEECF00F085
:1013DC00EDCF01F000C08DF001C08EF0140EE124B1
:1013EC00E96E000EE220EA6EEECF8FF0EECF90F0B9
:0413FC00EECF91F0AF
:10140000EDCF92F0ED52ED52180EE124E96E000E90
:10141000E220EA6EEECF93F0EECF94F0EECF95F0AF
:10142000EDCF96F0ED52ED52110EE8CF97F0FF0E92
:10143000E8CF98F00001996B9A6B98DB80C0E1FFD0
:1014400081C0E2FF140EE124E96E000EE220EA6E94
:10145000EE2A000EEE22EE22ED22ED52ED52050EA6
:10146000E76E1200D96E220D100EF324E16E010E0C
:10147000F420E26E0F0EE124E96E000EE220EA6E27
:10148000EF50006E0028D8B4000C210EE124E96E64
:10149000000EE220EA6EEF50006E00A2000C010E7A
:1014A000E124E8CF89F0000EE220E8CF8AF00B0EAD
:1014B000E124E96E000EE220EA6EEECF00F0EDCFFF
:1014C00001F000C08BF001C08CF00D0EE124E96E3C
:1014D000000EE220EA6EEECF00F0EDCF01F000C08A
:1014E0008DF001C08EF0140EE124E96E000EE220B2
:1014F000EA6EEECF8FF0EECF90F0EECF91F0EDCF21
:1015000092F0ED52ED52180EE124E96E000EE22049
:10151000EA6EEECF93F0EECF94F0EECF95F0EDCFF4
:1015200096F0ED52ED52100EE8CF97F00F0EE12439
:10153000E96E000EE220EA6EEF50E8CF98F0100E50
:10154000E124E96E000EE220EA6EEECF00F0EDCF6E
:1015500001F000C099F001C09AF0E1CF87F0E2CF2E
:1015600088F004DB87C0E1FF88C0E2FF140EE124AD
:10157000E96E000EE220EA6EEECF0CF1EECF0DF137
:10158000EECF0EF1EDCF0FF1ED52ED52100EE12442
:10159000E96E000EE220EA6EEECF00F0EDCF01F032
:1015A00000C002F101C003F1100EE124E96E000E4B
:1015B000E220EA6EEECF00F0EDCF01F0140EE12450
:1015C000E96E000EE220EA6E0050EE260150EE2297
:1015D000000EEE22ED22ED52ED52140EE124E96EE2
:1015E000000EE220EA6EEECF0CF1EECF0DF1EECF61
:1015F0000EF1EDCF0FF1ED52ED52210EE124E96E27
:10160000000EE220EA6EEF50FD0BEF6E210EE1249A
:10161000E96E000EE220EA6EEF50EF0BEF6E000174
:101620000F0E8725E96E000E8821EA6EEF503AEC26
:1016300024F087C0E1FF88C0E2FF0F0EE124E96ECD
:10164000000EE220EA6EFF0EEF6E210EE124E96E3D
:10165000000EE220EA6EEF50FD0B0209EF6E010C66
:10166000D96E220D1F0EF324E96E010EF420EA6EEE
:10167000EF50006E0028D8B436EF23F0D950220D79
:10168000310EF324E96E010EF420EA6EEF30010B07
:1016900012008300D96E220D100EF3240001856F15
:1016A000010EF420866FD950846F0F0E8525E96EE8
:1016B000000E8621EA6EEF50006E0028D8A427D0D5
:1016C0000F0E8525E96E000E8621EA6EEF6A0F0E79
:1016D0008525E96E000E8621EA6EEF5064EC24F059
:1016E0000001100E8525E96E000E8621EA6EEE6A75
:1016F000ED6A0001280EC16FC26B00010F0E852537
:10170000E96E000E8621EA6EEF505FEC24F00001D6
:10171000100E8525E96E000E8621EA6EEECFF3FFEE
:10172000EDCFF4FF000EF45CC40ED8B4F35CD8B077
:10173000000C210E8525E96E000E8621EA6EEF5021
:10174000EF0B1009EF6E8351E9EC23F085C0E1FF48
:1017500086C0E2FF100EE124E96E000EE220EA6E80
:10176000EECFF3FFEDCFF4FFF34AF42A100EE1249D
:10177000E96E000EE220EA6EF3CFEEFFF4CFEDFF4C
:10178000000EF45CC40ED8B4F35CD8A0010C0001C8
:10179000845168DE010CD96E220D100EF324E16E27
:1017A000010EF420E26EE1CF82F0E2CF83F0210E51
:1017B000E124E96E000EE220EA6EEF50006E00A612
:1017C000000CC6EC23F00001210E8225E96E000E0C
:1017D0008321EA6EEF50F70BEF6E010C1900D96E02
:1017E000220D100EF324E16E010EF420E26E210EA4
:1017F000E124E96E000EE220EA6EEF50006E00A6D2
:1018000033D0E1CF19F0E2CF1AF0210EE124E96ED6
:10181000000EE220EA6EEF50006E00A410D000012E
:10182000280E836F846B43EC24F00001210E1925F0
:10183000E96E000E1A21EA6EEF50FB0BEF6E00010D
:10184000210E1925E96E000E1A21EA6EEF50EF0BFA
:101850001009EF6E19C059F01AC05AF01BC05BF0A6
:101860001CC05CF0ACEF23F0006A016A12007F003C
:10187000D96E220D100EF324E16E010EF420E26EFB
:10188000210EE124E96E000EE220EA6EEF50006EB8
:1018900000A6000CE1CF81F0E2CF82F0210EE1241E
:1018A000E96E000EE220EA6EEF50006E00A410D048
:1018B0000001280E836F846B43EC24F00001210E9D
:1018C0008125E96E000E8221EA6EEF50FB0BEF6E70
:1018D0000001120E8125E96E000E8221EA6EEE50A3
:1018E000ED10D8A40DD0C6EC23F00001210E812507
:1018F000E96E000E8221EA6EEF50F70BEF6E000CDE
:101900000001120E8125E96E000E8221EA6EEE06BC
:10191000000EED5A82EC23F07FC0E9FF80C0EAFFA1
:10192000EF6E010CD96E220D310EF324E96E010E1B
:10193000F420EA6EEF30006E00320030010B12002E
:1019400012001F000001320E596F000E5A6F000185
:10195000140E5B6F5C6BACEC23F00001320EC16FB8
:10196000000EC26F32DB0001060E1F25E96E000E6D
:101970002021EA6EEECF26F0EECF27F0EECF28F052
:10198000EDCF29F0ED52ED5232C22AF033C22BF0E6
:1019900034C22CF035C22DF02E6B060EE8CF2FF09E
:1019A00021C030F022C031F030C0DCF031C0DDF0B9
:1019B00021EC26F000C030F001C031F00001260E0D
:1019C000DA6F000EDB6F00010C0EDC6FDD6B8AEC52
:1019D00026F0001C026E011C036E02C024F003C03E
:1019E00025F00001240E836F846B43EC24F0240E59
:1019F000E96E000EEA6EEF50E9EC23F0250EE96E79
:101A0000000EEA6EEF50E9EC23F00001140E836F34
:101A1000846B43EC24F021C0C1F022C0C2F0B2D9E3
:101A200000C024F001C025F0420EE96E000EEA6EFF
:101A30000001EE522551ED18D8B424C0E8FFEF188C
:101A4000D8B403D0C6EC23F0010C00013E390F0BD3
:101A5000006ED8900036D8900034EC0FD96E215D1E
:101A6000006E2251D8A02205016EEC0E0024216FD9
:101A7000FF0E0120226F3E390F0B006E016AD890D5
:101A800000360136D89000360136140E0024E8CF17
:101A900083F0000E0120E8CF84F043EC24F0000135
:101AA000320E466F000E476F1FC048F020C049F04D
:101AB000BBD90001236FFE0E235DD8A045D0C6EC34
:101AC00023F000012329D8A4010C21C000F022C07A
:101AD00001F0026A036A00503A2701503B2302508A
:101AE0003C2303503D233FB302D03FA106D0000169
:101AF0003A2B000E3B233C233D231FC089F020C01E
:101B00008AF034C08BF035C08CF032C08DF033C019
:101B10008EF03AC08FF03BC090F03CC091F03DC0D9
:101B200092F036C093F037C094F038C095F039C0C9
:101B300096F0040EE8CF97F0FF0EE8CF98F0000182
:101B4000996B9A6B13D8010C1FC046F020C047F068
:101B50000001320E486F000E496F21C04AF022C0CA
:101B60004BF0000123517CDB010C890036EC23F0A3
:101B70000009D8B4FBD78BC0ADF08CC0AEF08DC0DF
:101B8000AFF08EC0B0F08FC0B1F090C0B2F091C095
:101B9000B3F092C0B4F093C0B5F094C0B6F095C065
:101BA000B7F096C0B8F00001BA513F0BBA6FB95107
:101BB000F00BB96F97C0BAF065EC24F000C0BBF031
:101BC00001C0BCF00001000EBC5D290ED8B4BB5DA5
:101BD000D8A005D0D80EBB27FF0EBC2303D0000130
:101BE000BB6BBC6B0001BD6BBE6BBF6BC06B000100
:101BF000AD0EC16F000EC26FE8D9140E0001992717
:101C0000000E9A2397A312D0040E9927000E9A2350
:101C1000020EE8CF9DF0040EE8CF9EF09F6BFA0E07
:101C2000E8CFA0F0B9510F0B600904D00001B95101
:101C30000F0B5009B96F32C2A1F033C2A2F034C207
:101C4000A3F035C2A4F00001060E8925E96E000E4E
:101C50008A21EA6EEECFA5F0EECFA6F0EECFA7F088
:101C6000EDCFA8F0ED52ED52A96B060EE8CFAAF029
:101C700099C0ABF09AC0ACF0ABC0DCF0ACC0DDF00A
:101C800021EC26F000C0ABF001C0ACF00001A10EC9
:101C9000DA6F000EDB6F00010C0EDC6FDD6B8AEC7F
:101CA00026F0001C026E011C036E02C0BDF003C0D2
:101CB000BEF0BD0EE96E000EEA6EEECF9BF0EDCFEA
:101CC0009CF000019829D8B4986B0001140EC16FE4
:101CD000C26B000198515FEC24F089C0C1F08AC04A
:101CE000C2F0060EE8CFC3F099C0C4F09AC0C5F0A8
:101CF00061EC25F00001AD0EDA6F000EDB6F000124
:101D0000140EDC6FDD6B13EC24F097A30BD00001F5
:101D10009D0EDA6F000EDB6F0001040EDC6FDD6BD1
:101D200013EC24F00001140EC16FC26B0001985136
:101D30005FEC24F099C0C1F09AC0C2F023D800C073
:101D40009BF001C09CF00001240EC16FC26B00012A
:101D500098515FEC24F09C0EE96E000EEA6EEF5095
:101D6000E9EC23F09B0EE96E000EEA6EEF50E9EC11
:101D700023F00001C16BC26B000198515FEC24F0AD
:101D80002FEF24F00001C36BC32BC56BC66B0001A2
:101D9000C251016EC151006EC107D8A0C207011027
:101DA000D8B42CD082EC23F00001C46FC351D8A466
:101DB0000FD0C451C525E8CFC5F0C451C5C000F04F
:101DC000005CD8B014D0C63F12D00001C52B0FD094
:101DD0000001C451C625E8CFC6F0C451C6C000F00A
:101DE000005CD8B004D0C53F02D00001C62B000172
:101DF000C351000ED8B4010EC36FC9D7C60EE96E29
:101E0000000EEA6EEF50FF0AE8CFC6F0C50EE96E8D
:101E1000000EEA6EEF50FF0AE8CFC5F0C5C000F033
:101E2000C6C001F0120046000001FE0E4A6F016AB2
:101E30000150220D100EF324D96E010EF420DA6E3B
:101E4000DF50D8B44ED00001020E4625E16E000EE0
:101E50004721E26E0B0ED924E96E000EDA20EA6EFD
:101E6000EE52E652E550ED18E7CFE8FFD8B4EF1890
:101E7000D8A437D0DF50006E0004D8A402D001509F
:101E80004A6F46C0E9FF47C0EAFF0D0ED924E16E54
:101E9000000EDA20E26EE652EE52ED50E518EFCF7A
:101EA000E8FFD8B4E718D8A41CD00001060E4825D6
:101EB000E16E000E4921E26E070ED924E96E000E94
:101EC000DA20EA6EEE50E61808E1EE50E61805E179
:101ED000EE50E61802E1EE50E618D8A402D0015008
:101EE0001200012A070E015CD8A0A2D700014A51B6
:101EF000220D100EF324E16E010EF420E26E4A5121
:101F0000FE0AD8B45BD0E750006E0004D8A456D0C7
:101F1000010EE124E8CF5FF0000EE220E8CF60F090
:101F2000E1CF4BF0E2CF4CF048C061F049C062F025
:101F300000010A0E636F646B8AEC2CF04BC0D9FF72
:101F40004CC0DAFF0001020E4625E16E000E47216B
:101F5000E26E0B0ED924E96E000EDA20EA6EE6CFAF
:101F6000EEFFE5CFEDFF46C0E9FF47C0EAFF0D0EEB
:101F7000D924E16E000EDA20E26EEECFE6FFEDCF5F
:101F8000E5FF210ED924E96E000EDA20EA6EEF504B
:101F9000F70BEF6E0F0ED924E96E000EDA20EA6E11
:101FA000FF0EEF6E210ED924E96E000EDA20EA6EE4
:101FB000EF50FD0B0209EF6E4A51120000014A5129
:101FC000FE0AD8B4FF0CFE0CC100C1C0E9FFC2C0BC
:101FD000EAFFEECF00F0EDCF01F000C0DCF001C071
:101FE000DDF021EC26F0C1C0E9FFC2C0EAFF00C06D
:101FF000EEFF01C0EDFF0001020EC125E96E000EEB
:10200000C221EA6EEECF00F0EDCF01F000C0DCF0AF
:1020100001C0DDF021EC26F00001020EC125E96EC1
:10202000000EC221EA6E00C0EEFF01C0EDFF040EFB
:10203000C125E96E000EC221EA6EEECFC3F0EECFED
:10204000C4F0EECFC5F0EDCFC6F0ED52ED5238EC56
:1020500026F00001040EC125E96E000EC221EA6ED1
:1020600000C0EEFF01C0EEFF02C0EEFF03C0EEFFB6
:10207000080EC125E96E000EC221EA6EEECFC3F054
:10208000EECFC4F0EECFC5F0EDCFC6F0ED52ED527D
:1020900038EC26F00001080EC125E96E000EC221C1
:1020A000EA6E00C0EEFF01C0EEFF02C0EEFF03C00B
:1020B000EEFF0E0EC125E96E000EC221EA6EEECFD4
:1020C00000F0EDCF01F000C0DCF001C0DDF021EC4C
:1020D00026F000010E0EC125E96E000EC221EA6E47
:1020E00000C0EEFF01C0EDFF100EC125E96E000E2D
:1020F000C221EA6EEECF00F0EDCF01F000C0DCF0BF
:1021000001C0DDF021EC26F00001100EC125E96EC2
:10211000000EC221EA6E00C0EEFF01C0EDFF120EFC
:10212000C125E96E000EC221EA6EEECF00F0EDCFC0
:1021300001F000C0DCF001C0DDF021EC26F0000170
:10214000120EC125E96E000EC221EA6E00C0EEFF3C
:1021500001C0EDFF1200820000010F0E8225E96E22
:10216000000E8321EA6EEF50006E0028D8B41FD015
:102170000F0E8225E96E000E8321EA6EEF503AECD5
:1021800024F082C0E1FF83C0E2FF0F0EE124E96E7C
:10219000000EE220EA6EFF0EEF6E210EE124E96EE2
:1021A000000EE220EA6EEF50FD0B0209EF6E82C0D6
:1021B000E1FF83C0E2FF070EE124E96E000EE2209A
:1021C000EA6EEE6AEE6AEE6AED6AED52ED520D0EBF
:1021D000E124E96E000EE220EA6E000EEE6AED6A7E
:1021E000E1CF82F0E2CF83F0210EE124E96E000E10
:1021F000E220EA6EEF50006E00B6C6EC23F082C01B
:10220000E1FF83C0E2FF210EE124E96E000EE2202F
:10221000EA6EEF50F70BEF6E1F0EE124E96E000E31
:10222000E220EA6E580EEE6E020EED6E210EE124F3
:10223000E96E000EE220EA6EEF50EF0BEF6E210E1A
:10224000E124E96E000EE220EA6EEF50006E00A07D
:1022500003D0010EE76E1200000EE76A120046007E
:10226000D96E00014C6BD950220D100EF324E16E93
:10227000010EF420E26E180EE124E96E000EE22059
:10228000EA6EEECF4FF0EECF50F0EECF51F0EECF42
:1022900052F0140EE124E96E000EE220EA6EEECF59
:1022A00053F0EECF54F0EECF55F0EECF56F0040ED3
:1022B0004825E96E000E4921EA6EEECF5BF0EECFC5
:1022C0005CF0EECF5DF0EECF5EF04AC000F04BC0A8
:1022D00001F0026A036A00505B2701505C23025040
:1022E0005D2303505E23140EE124E96E000EE2200C
:1022F000EA6EEECF57F0EECF58F0EECF59F0EECFBA
:102300005AF0080E4825E96E000E4921EA6EEECF1C
:1023100008F1EECF09F1EECF0AF1EDCF0BF1ED525E
:10232000ED521C0EE124E96E000EE220EA6E000E72
:10233000EF6AE1CF4DF0E2CF4EF04BEC2DF0000113
:102340001D0E4D25E96E000E4E21EA6E00C0EEFF17
:1023500001C0EDFF4DC0D9FF4EC0DAFF1F0ED924DA
:10236000E96E000EDA20EA6E580EEE6E020EED6E89
:10237000DF50006E0004D8A4A5D0C6EC23F04DC0F9
:10238000D9FF4EC0DAFF0101042B000E05230623FE
:102390000723140ED924E96E000EDA20EA6E04C178
:1023A000EEFF05C1EEFF06C1EEFF07C1EEFF000123
:1023B0005B2B000E5C235D235E23180ED924E96E8F
:1023C000000EDA20EA6E5BC0EEFF5CC0EEFF5DC07F
:1023D000EEFF5EC0EEFF140ED924E96E000EDA2087
:1023E000EA6EEECF57F0EECF58F0EECF59F0EECFC9
:1023F0005AF0140ED924E96E000EDA20EA6EEE2AA5
:10240000000EEE22EE22ED22ED52ED5248C0E1FF29
:1024100049C0E2FF0D0EE124E96E000EE220EA6EF3
:10242000EF50006E00A229D0010ED924E8CF5FF052
:10243000000EDA20E8CF60F046C061F047C062F0DD
:1024400000010A0E636F646B8AEC2CF04DC0D9FF5B
:102450004EC0DAFF48C0E9FF49C0EAFF0D0ED9249B
:10246000E16E000EDA20E26EEECFE6FFEDCFE5FF83
:102470000001120E4C6F020E62D20001040E4C6F6E
:102480005BC057F05CC058F05DC059F05EC05AF0B8
:10249000E124E96E000EE220EA6EEECF5BF0EECFB3
:1024A0005CF0EECF5DF0EECF5EF0070ED924E96E62
:1024B000000EDA20EA6EEE6AEE6AEE6AED6AED521E
:1024C000ED5259D248C0E1FF49C0E2FF0D0EE124B0
:1024D000E96E000EE220EA6EEF50006E00A407D015
:1024E000C6EC23F04DC082F04EC083F035D6080E06
:1024F000E124E96E000EE220EA6E0001EE50571969
:1025000008E1EE50581905E1EE50591902E1EE507C
:102510005A19D8A42ED2DF50020AD8A457D00D0ED3
:10252000E124E96E000EE220EA6EEF50006E00A892
:102530004AD0180ED924E96E000EDA20EA6E5BC08C
:10254000EEFF5CC0EEFF5DC0EEFF5EC0EEFF1C0E56
:10255000D924E96E000EDA20EA6E000EEF6A4BEC29
:102560002DF000011D0E4D25E96E000E4E21EA6E84
:1025700000C0EEFF01C0EDFF4DC0E1FF4EC0E2FF25
:10258000040EE76E4B514A11D8B41AD0210EE12443
:10259000E96E000EE220EA6EEF50F70B0809EF6ECD
:1025A000120EE124E96E000EE220EA6E4AC0EEFF50
:1025B0004BC0EDFF210EE124E96E000EE2206DD04C
:1025C000C6EC23F0D8D1C6EC23F0D5D1DF50030AF6
:1025D000D8A46FD00D0EE124E96E000EE220EA6E61
:1025E000EF50006E00A262D000015B2B000E5C2356
:1025F0005D235E23180ED924E96E000EDA20EA6E00
:102600005BC0EEFF5CC0EEFF5DC0EEFF5EC0EEFFA4
:102610000D0EE124E96E000EE220EA6EEF50006E2E
:1026200000A805D0100E4C6F040EDF6E18D000010C
:10263000120E4C6F020EDF6E572B000E58235923DB
:102640005A23140ED924E96E000EDA20EA6E57C020
:10265000EEFF58C0EEFF59C0EEFF5AC0EEFF00017A
:102660004B514A11D8B41FD0210ED924E96E000E67
:10267000DA20EA6EEF50F70B0809EF6E120ED9243C
:10268000E96E000EDA20EA6E4AC0EEFF4BC0EDFFA5
:10269000210ED924E96E000EDA20EA6EEF50FB0B12
:1026A0000409EF6E68D1C6EC23F065D1C6EC23F0C7
:1026B00062D1180ED924E16E000EDA20E26E00011C
:1026C000040E4825E96E000E4921EA6EEE50E61828
:1026D00008E1EE50E61805E1EE50E61802E1EE5092
:1026E000E618D8A4C6EF23F0180ED924E96E000E20
:1026F000DA20EA6E5BC0EEFF5CC0EEFF5DC0EEFF6D
:102700005EC0EEFFDF50040AD8A4BFD000010D0E5A
:102710004825E96E000E4921EA6EEF50006E00A8D0
:102720002AD00F0ED924E96E000EDA20EA6EEF509F
:10273000006E0028D8B41FD00F0E4D25E96E000E94
:102740004E21EA6EEF503AEC24F04DC0D9FF4EC056
:10275000DAFF0F0ED924E96E000EDA20EA6EFF0EC2
:10276000EF6E210ED924E96E000EDA20EA6EEF50EA
:10277000FD0B0209EF6E00010D0E4825E96E000EFB
:102780004921EA6EEF50006E00A02BD0110E4C6F65
:10279000140ED924E96E000EDA20EA6E5DEC2DF0FD
:1027A00000C057F001C058F002C059F003C05AF001
:1027B000180ED924E96E000EDA20EA6EEE2A000E19
:1027C000EE22EE22ED22ED52ED52EECF5BF0EECF97
:1027D0005CF0EECF5DF0EDCF5EF0ED52ED520A0E03
:1027E000DF6E00014B514A11D8B44CD0210ED924D0
:1027F000E96E000EDA20EA6EEF50006E00B621D0CE
:10280000210ED924E96E000EDA20EA6EEF50F70BA4
:102810000809EF6E120ED924E96E000EDA20EA6E76
:102820004AC0EEFF4BC0EDFF210ED924E96E000E29
:10283000DA20EA6EEF50FB0B0409EF6E100E4C6FBE
:102840009AD000014C6B140ED924E96E000EDA20E8
:10285000EA6E53C0EEFF54C0EEFF55C0EEFF56C007
:10286000EEFF180ED924E96E000EDA20EA6E4FC092
:10287000EEFF50C0EEFF51C0EEFF52C0EEFFC6ECBF
:1028800023F079D0C6EC23F076D0DF500A0AD8A422
:1028900013D0C6EC23F000010D0E4825E96E000EA2
:1028A0004921EA6EEF50006E00A865D04DC082F05D
:1028B0004EC083F051DC5FD0DF50050AD8A441D070
:1028C000C6EC23F048C0E1FF49C0E2FF0D0EE12451
:1028D000E96E000EE220EA6EEF50006E00A04BD0D1
:1028E0000001100E4C6F4DC0D9FF4EC0DAFF180E1C
:1028F000D924E96E000EDA20EA6EEE2A000EEE22EE
:10290000EE22ED22ED52ED52EECF5BF0EECF5CF019
:10291000EECF5DF0EDCF5EF0ED52ED520D0EE12405
:10292000E96E000EE220EA6EEF50006E00A806D0BD
:10293000D9CF82F0DACF83F00FDC1DD0060EDF6E28
:102940001AD0DF50060AD8A416D0C6EC23F0000136
:102950000D0E4825E96E000E4921EA6EEF50006E1B
:1029600000A809D04DC082F04EC083F0ACEC10F04E
:1029700002D0C6EC23F000014C51D8B4120046C07E
:1029800089F047C08AF048C0E1FF49C0E2FF020E6B
:10299000E124E96E000EE220EA6EEECF00F0EDCF0A
:1029A00001F000C08BF001C08CF0E6CF00F0E5CF65
:1029B00001F000C08DF001C08EF057C08FF058C0FC
:1029C00090F059C091F05AC092F05BC093F05CC097
:1029D00094F05DC095F05EC096F04CC097F0FF0E8D
:1029E000E8CF98F00001996B9A6BB6EF0DF00001FB
:1029F000196B0001500E1A6F1B6B49EC09F0006E49
:102A0000000119510A0D000EF324E96E020EF420A4
:102A1000EA6E00C0EFFF19510A0D030EF324E96EB0
:102A2000020EF420EA6EEF6A192B050E195DD8B07C
:102A30001200DFD70001196B0001195107D80001FE
:102A4000192B050E195DD8B01200F6D7D96E0A0DF4
:102A5000000EF3240001226F020EF420236F1B6B83
:102A60001B2B00011B51D8B412001B6B22C0E9FFC5
:102A700023C0EAFFEF50A2EC09F000090001030EA9
:102A8000D8A411D22225E96E000E2321EA6E000E91
:102A9000EF6A120022C0E9FF23C0EAFFEF5092EC78
:102AA0000CF000090001D8B4DDD71B6B1B2B1E6B8B
:102AB0001F6B0001000E1F5D500ED8B41E5DD8B014
:102AC0001AD01F51016E1E51006E1E4B1F2B2E0F70
:102AD000E8CF7FF0000E0120E8CF80F022C0E9FFB0
:102AE00023C0EAFFEF5038EC0CF0006E016A015091
:102AF0000010D8A4DED700012E0E1E25E96E000EB0
:102B00001F21EA6E000EEF6A22C0E9FF23C0EAFF30
:102B1000EF50CBEC0BF00001030E2225E96E000E06
:102B20002321EA6E020EEF6E050E1C6F00012E0EC1
:102B30007F6F000E806F0001240E816F000E826F88
:102B400000011C0E836F000E846F0001090E222508
:102B5000E8CF85F0000E2321E8CF86F0C5DA00012A
:102B60001A6F0009D8A47DD7020E1C5DD8A012D020
:102B70000001240E7F6F000E806F1CC081F0FDEC01
:102B80001BF00001090E2225E96E000E2321EA6EDA
:102B9000030EEF6E24C07FF025C080F0BFEC28F05C
:102BA0000001010E2225E96E000E2321EA6E00C00D
:102BB000EEFF01C0EDFF22C0E1FF23C0E2FF010EE6
:102BC000E124E96E000EE220EA6EEE52ED50FF0ABB
:102BD000FF0ED8B4EF18D8A411D0080EE124E96E86
:102BE000000EE220EA6E000EEF6E030EE124E96EA5
:102BF000000EE220EA6E020EEF6E33D7010EE124E2
:102C0000E96E000EE220EA6EEE50ED10D8A408D076
:102C1000080EE124E96E000EE220EA6E030EE4D70E
:102C2000030EE124E96E000EE220EA6E0B0EE4D7FB
:102C300022C0E9FF23C0EAFFEF5030EC0BF000099F
:102C40000001D8B40FD7080E2225E96E000E23210B
:102C5000EA6EEF50006E016AD8900034026E0134C3
:102C6000036EE80E0224E96E000E0320EA6EEECF3A
:102C700020F0EDCF21F0000120C0F6FF21C0F7FFCA
:102C8000010E2027000E2123050EF76403D0080053
:102C9000F55005D0F6CFE9FFF7CFEAFFEF50D96E38
:102CA0000009D8B40AD0D9CF83F022C0E9FF23C0ED
:102CB000EAFFEF504AEC0BF0DED722C0E9FF23C059
:102CC000EAFFEF5032EC0AF0C1D022C0E9FF23C086
:102CD000EAFFEF5030EC0BF000090001D8B4C2D687
:102CE0001B6B1B2B1D6B1D51006E016A0050A80F42
:102CF000F66E0150F76E060EF7220800F550E8CF89
:102D000083F022C0E9FF23C0EAFFEF504AEC0BF04A
:102D100000011D2B1F0E1D5DD8A0E5D7090E222531
:102D2000E96E000E2321EA6EEF50140D1C0EF32401
:102D3000206F060EF420216F000120C0F6FF21C095
:102D4000F7FF010E2027000E2123050EF76403D0A4
:102D50000800F55005D0F6CFE9FFF7CFEAFFEF50B6
:102D6000D96E0009D8B40AD0D9CF83F022C0E9FFC8
:102D700023C0EAFFEF504AEC0BF0DED700011D6BD9
:102D800000011D51006E016A0050C80FF66E01501F
:102D9000F76E060EF7220800F550E8CF83F022C048
:102DA000E9FF23C0EAFFEF504AEC0BF000011D2BB6
:102DB000040E1D5DD8A0E4D722C0E1FF23C0E2FFCE
:102DC000090EE124E96E000EE220EA6EEF50030ADC
:102DD000070ED8A407D0E124E96E000EE220EA6EC7
:102DE000010E06D0E124E96E000EE220EA6E000E2C
:102DF000EF6E040EE124E96E000EE220EA6E030E8F
:102E0000EF6EE124E96E000EE220EA6E010EF4D6C8
:102E100022C0E9FF23C0EAFFEF5092EC0CF000095A
:102E2000D8B407D022C0E9FF23C0EAFFEF50CBECB3
:102E30000BF022C07FF023C080F048D8006E016AFA
:102E400001500010D8B40DD65FEC29F00001030E3C
:102E50002225E96E000E2321EA6E090ECDD622C08E
:102E6000E9FF23C0EAFFEF50A2EC09F00009D8B453
:102E7000F8D522C0E9FF23C0EAFFEF5030EC0BF099
:102E80000009D8B4EED522C0E9FF23C0EAFFEF5015
:102E9000B0EC09F00001030E2225E96E000E23219B
:102EA000EA6E0A0EA9D62225E96E000E2321EA6EEB
:102EB000EF5001E1EFD5010AABE0030A01E1B8D61A
:102EC0000B0ACDE0020A01E100D7CBD50001010ECB
:102ED0007F25E96E000E8021EA6EEECF00F0EDCF87
:102EE00001F000C0FEF101C0FFF1B1D0000182513C
:102EF000250AD8A408D0040EE124E96E000EE220D1
:102F0000EA6E050E12D00001816B812B93D0000177
:102F10008251250AD8A40BD0816B812B040EE124A9
:102F2000E96E000EE220EA6E030EEF6E83D0080E0B
:102F3000E124E96E000EE220EA6E82C000F0D00EBD
:102F400000260038F00BEF6E040EE124E96E000E4F
:102F5000E220EA6E060EE9D782C000F0D00E00260D
:102F6000080EE124E96E000EE220EA6E0050EF1236
:102F7000040EE124E96E000EE220EA6E080EEF6E08
:102F8000050EE124E96E000EE220EA6EEE6AED6ABB
:102F900051D00001050E7F25E96E000E8021EA6EFA
:102FA000EECF00F0EDCF01F000C083F001C084F05F
:102FB0000001820E856F000E866F0001080E7F25CE
:102FC000E96E000E8021EA6EEF5051EC1CF000011A
:102FD000050E7F25E96E000E8021EA6E00C0EEFF2F
:102FE00001C0EDFF816B812B7FC0E1FF80C0E2FF5C
:102FF000050EE124E96E000EE220EA6EEE52ED507D
:10300000FF0AFF0ED8B4EF18D8A414D087D7FFD783
:10301000040EE124E96E000EE220EA6EEF50030A8E
:1030200001E164D7060A01E172D7030A95E00E0AAE
:10303000B0E0EDD700018151D8B409D082C083F04F
:103040007FC0E9FF80C0EAFFEF504AEC0BF07FC081
:10305000E9FF80C0EAFFEF5030EC0BF000090001FF
:10306000D8B436D0816B040E7F25E96E000E802126
:10307000EA6EEF50080AD8B414D074EC29F00001BD
:10308000826F0101FF51FF0AFF0ED8B4FE19D8A4C8
:1030900008D07FC0E9FF80C0EAFFEF5032EC0AF0B1
:1030A000010C7FC0E1FF80C0E2FF070EE124E96E62
:1030B000000EE220EA6EEF50D8A4AAD782C083F0B7
:1030C0007FC0E9FF80C0EAFFEF504AEC0BF0BFD7AA
:1030D000010E7F25E96E000E8021EA6EFEC1EEFF33
:1030E000FFC1EDFF000C7F000001886B8D6B8E6BC4
:1030F000896B7FC08FF080C090F00001CD0E916F82
:10310000060E926F0001030E936F946B37EC2CF058
:1031100001500010D8A40BD07FC0E1FF80C0E2FFB7
:10312000040EE126000EE2220001876B21D07FC051
:103130008FF080C090F00001D10E916F060E926F5B
:103140000001040E936F946B37EC2CF001500010CB
:10315000D8A4020C7FC0E1FF80C0E2FF050EE1268B
:10316000000EE2220001876B872B02D0E14AE22A9F
:10317000E750200AD8B4FAD7A0D083C0E9FF84C0B2
:10318000EAFFEF500001895DD8B0A7D088D00001D8
:103190008951006E016AD8900034026E0134036ECA
:1031A000D9500224E96EDA500320EA6EE1CFEEFF37
:1031B000E2CFEDFFE7CFF3FFF3502F0AD8B429D0C9
:1031C000F3505C0AD8A477D024D000018951006E56
:1031D000016AD8900034026E0134036ED950022483
:1031E000E96EDA500320EA6EE1CFEEFFE2CFEDFFA9
:1031F000892B020E886F5FD0E7CFF3FFF3503F0AB1
:10320000D8B404D0F350260AD8A406D0000EE76A3A
:103210000001886B882B4FD0F3502B0AD8A403D021
:10322000200EE76E48D0F3502E0AD8A410D000012B
:103230008905D8A40CD0E10EE96E0F0EEA6EEE2AD5
:10324000000EED22EECF8DF0EDCF8EF034D0F350A6
:103250003D0AD8B4DBD7F3502F0AD8B404D0F350CA
:103260005C0AD8A428D000018951006E016AD89068
:103270000034026E0134036ED9500224006EDA501D
:103280000320016EFE0E0024E96EFF0E0120EA6E9F
:10329000010EE124EE6E000EE220ED6E0CD081C036
:1032A000D9FF82C0DAFF0001885101E170D7010A1D
:1032B0008CE0030AA1E0E14AE22AE7CFD9FFD95026
:1032C000200AD8B40AD0D950D8B407D00D0AD8B43F
:1032D00004D0D9500A0AD8A450D7000EE76A85C096
:1032E000E9FF86C0EAFF070EEF6E00018E518D11D7
:1032F000D8B433D08DC093F08EC094F015EC27F085
:1033000000C08DF001C08EF00001000E8B6F060E24
:103310008C6F8A6B8DC08FF08EC090F08BC091F057
:103320008CC092F00001030E936F946B37EC2CF07D
:1033300001500010D8A407D085C0E9FF86C0EAFF7D
:103340008AC0EFFF0AD0040E00018B27000E8C23E9
:103350008A2B070E8A5DD8A0DDD700018951D8A439
:103360002ED081C0E9FF82C0EAFFEECF00F0EDCFA2
:1033700001F000C093F001C094F00001D60E956FEB
:10338000060E966F090EE8CF97F046EC27F081C045
:10339000E9FF82C0EAFFEECF00F0EDCF01F0090EA9
:1033A0000024E96E000E0120EA6E000EEF6A85C06F
:1033B000E9FF86C0EAFF010EEF6E0001892B83C092
:1033C000E9FF84C0EAFF89C0EFFF000187511200C6
:1033D00050EC2DF0B1EC21F0E2C5F3FFE3C5F4FFB2
:1033E000E4C5F5FFE5C5F6FFE6C5F7FFE7C5F8FF5D
:1033F000E8C500F0E9C501F0EAC502F0EBC503F04D
:10340000ECC504F0EDC505F0EEC506F0EFC507F01C
:10341000F0C508F0F1C509F0F2C50AF0F3C50BF0EC
:10342000F4C50CF0F5C50DF0F6C50EF0F7C5DAFFE2
:10343000F8C5D9FFF9C5E2FFFAC5E1FFFBC5EAFF10
:10344000FCC5E9FFFDC5E8FFFEC5FAFFFFC5D8FFD3
:103450000FC0E0FF1000E0CF0FF0E8CFFDF5E9CF9F
:10346000FCF5EACFFBF5E1CFFAF5E2CFF9F5D9CFDC
:10347000F8F5DACFF7F50EC0F6F50DC0F5F50CC08E
:10348000F4F50BC0F3F50AC0F2F509C0F1F508C078
:10349000F0F507C0EFF506C0EEF505C0EDF504C088
:1034A000ECF503C0EBF502C0EAF501C0E9F500C098
:1034B000E8F5F8CFE7F5F7CFE6F5F6CFE5F5F5CF88
:1034C000E4F5F4CFE3F5F3CFE2F582D7ACA2FED773
:1034D000AD6E1200430043C0E1FF44C0E2FFE25082
:1034E000016EE150006EE14AE22A00C0E9FF01C02E
:1034F000EAFFEF50D96ED8B41200E8DFF0D7F86ACF
:103500004ADA41EC2DF0B5EC28F063DA81BA0BD041
:10351000C00E09EC2BF000010D0E436F0F0E446F2F
:1035200074EC2BF0FEDBD5EC29F0F7EC14F0DDECBD
:1035300029F01AEC15F00DD9D1C500F0AAC5E8FFA5
:103540000018D8B4F4D70001320E366F020E376F70
:10355000010EE8CF38F019D8AAC5D1F54AC200F05B
:1035600000A0E5D7CE0E09EC2BF00A0ED1C500F075
:10357000005CD1C5E8FFD8B004D0300F94EC2BF03C
:10358000D6D7410F94EC2BF0D2D700013851D8B4E4
:103590000DD0C00E09EC2BF000011C0E436F0F0E76
:1035A000446F74EC2BF0C00E09EC2BF00001390EC7
:1035B000456F000E466F0001E50E476F100E486F15
:1035C00036C0E9FF37C0EAFFEF50006E016A00C065
:1035D00041F001C042F0410EE8CF43F0000EE8CFC9
:1035E00044F0B1EC1EF000013851D8B40BD000010A
:1035F000390E436F000E446F5DEC2BF02E0E94ECF1
:103600002BF008D00001390E436F000E446F63DFCA
:103610002E0E5CDF0001390E456F000E466F000173
:10362000E50E476F100E486F0001010E3625E96E5A
:10363000000E3721EA6EEF50006E016A00C041F0C3
:1036400001C042F0410EE8CF43F0000EE8CF44F055
:10365000B1EC1EF000013851D8B40BD00001390E86
:10366000436F000E446F5DEC2BF02E0E94EC2BF0AC
:1036700008D00001390E436F000E446F2CDF2E0E70
:1036800025DF0001390E456F000E466F0001E50E83
:10369000476F100E486F0001020E3625E96E000ECE
:1036A0003721EA6EEF50006E016A00C041F001C0A0
:1036B00042F0410EE8CF43F0000EE8CF44F0B1EC09
:1036C0001EF000013851D8B40BD00001390E436F01
:1036D000000E446F5DEC2BF02E0E94EC2BF008D016
:1036E0000001390E436F000E446FF5DE2E0EEEDE44
:1036F0000001390E456F000E466F0001E50E476F61
:10370000100E486F0001030E3625E96E000E3721BA
:10371000EA6EEF50006E016A00C041F001C042F055
:10372000410EE8CF43F0000EE8CF44F0B1EC1EF0BC
:1037300000013851D8B407D00001390E436F000E94
:10374000446F5DEF2BF00001390E436F000E446FA4
:10375000C2D6810EC26E640EE8CF19F000011907BF
:103760001929D8A4FBD7C284C2B4FED7C3CF19F09D
:10377000C4CF1AF00001D20E456F050E466F00014E
:10378000E50E476F100E486F19C01BF01AC01CF0F1
:103790001B0EE8CF43F0000EE8CF44F0B1EC1EF072
:1037A000840EC16E890EC26E640EE8CF19F000015E
:1037B00019071929D8A4FBD7C284C2B4FED7C3CF36
:1037C00019F0C4CF1AF00001DA0E456F050E466FEE
:1037D0000001E50E476F100E486F19C01BF01AC0AC
:1037E0001CF01B0EE8CF43F0000EE8CF44F0B1EC24
:1037F0001EF08E0EC16E12007F007FC0E1FF80C000
:10380000E2FFE6CF00F0E5CF01F000C0E9FF01C024
:10381000EAFFEF50D00FD96E3FD0020EE124E96EDF
:10382000000EE220EA6EEECF00F0EDCF01F000C016
:10383000E9FF01C0EAFFEF50D00FD96E04D08976BE
:1038400006D0897404D0D950FAE0010AFAE0E6CF34
:1038500000F0E5CF01F000C093F001C094F000014A
:103860002D0E956F0F0E966F0D0EE8CF97F046EC6C
:1038700027F01200E6CF00F0E5CF01F000C093F092
:1038800001C094F000013A0E956F0F0E966F0A0E6C
:10389000E8CF97F046EF27F0D950BFE0010AE9E002
:1038A000E9D7E16E66D089B603D060D089A45ED036
:1038B000300E5DD0000184518311D8A402D0836BF7
:1038C000846BD20E006E050E016E00018351002440
:1038D000E96E000E0120EA6EEFCFDFFFD20E006E20
:1038E000050E016E83510024E96E000E0120EA6E80
:1038F000EF50D8A404D0FF0E006E016E120000013C
:10390000834B842B83C000F084C001F012000001BF
:1039100084518311D8A402D0836B846BDA0E006EBD
:10392000050E016E000183510024E96E000E012096
:10393000EA6EEFCFDFFFDA0E006E050E016E8351E7
:103940000024E96E000E0120EA6EEF50D8A404D0E6
:10395000FF0E006E016E12000001834B842B83C0AA
:1039600000F084C001F0120081AAA2D7310EDF6EF0
:103970000ED085C0D9FF86C0DAFFE15094E0010A7D
:1039800095E0030A97E0010AC2E0070AEDE0FF0EA6
:10399000006E016E12008E0EC16E030E926E809A42
:1039A00089848986F19ED0EC2AF0800E09EC2BF0F8
:1039B0000001FE0E436F0E0E446F74EC2BF0200ED0
:1039C000AC6E900EAB6E0F0EAF6ED56AF28EF28CAF
:1039D00012000A0EE8CF32F2E8CF33F2050EE8CF3C
:1039E00034F20F0EE8CF35F2FF0EE8CF3CF2E8CF0D
:1039F0003DF2E8CF3EF202013F6B0A0EE8CF40F203
:103A0000E8CF41F2050EE8CF42F20F0EE8CF43F2C5
:103A10000201366B040EE8CF37F2A30EE8CF38F27E
:103A20000201396B02013A6B02013B6B4A0EE96EEF
:103A3000020EEA6EEF50FE0BEF6E12003600000130
:103A400036C0F6FF37C0F7FF010E3627000E3723CA
:103A5000050EF76403D00800F55005D0F6CFE9FF56
:103A6000F7CFEAFFEF50D96E0009D8B412002EDD6F
:103A7000E6D736C0E1FF37C0E2FFD96A9EAAFED77B
:103A8000AE50F36E0D0AD8B40DD0F3500A0AD8B474
:103A900009D0D92AF3CFE6FFE76A000138073829B1
:103AA000D8A4ECD7D9501200360036C0E1FF37C099
:103AB000E2FFE1CF3BF0E2CF3CF000013A6BE75090
:103AC000D96ED8B437D02E0AD8A429D0E250016ECE
:103AD000E150006EE14AE22A00C0E9FF01C0EAFFBE
:103AE000000EEF6AE1CF36F0E2CF37F03BC03DF099
:103AF0003CC03EF016EC02F000013A513825E96E68
:103B0000000E3921EA6E00C0EFFF3A2B36C0E1FF0C
:103B100037C0E2FFE1CF3BF0E2CF3CF008D0300EFF
:103B2000D95CD8A0000C3A0ED95CD8B0000CE14AA0
:103B3000E22AC5D73BC03DF03CC03EF016EC02F097
:103B400000013A513825E96E000E3921EA6E00C0B5
:103B5000EFFF3A51030A000ED8B4010E12009EAADC
:103B6000FED7AE50D96E310ED95C390ED8A01200F6
:103B7000D95CD8B0390CD9501200E16E0D0EA6DC1C
:103B80000A0EA4DCE150006E016AD8900034026E87
:103B90000134036E8E0E0224E96E000E0320EA6EDD
:103BA000EECF00F0EDCF01F000C036F001C037F0ED
:103BB00046DFA4D00001200E456F000E466F0001C5
:103BC000E50E476F100E486F440EE96E020EEA6E66
:103BD000EECF34F0EDCF35F0340EE8CF43F0000EE9
:103BE000E8CF44F0B1EC1EF00001200E436F000E50
:103BF000446F71DC290E6ADC3A0E68DC200E66DC4C
:103C00000001200E366F000E376F140EE8CF38F02B
:103C100030DF006E016A01500010D8B447D00001B7
:103C2000200E3D6F000E3E6F16EC02F000C044F215
:103C300001C045F245C23AF244C23BF21200320ED4
:103C4000E96E020E07D0400EE96E020E03D03C0E64
:103C5000E96E020EEA6EE9CF36F0EACF37F0E9CF2F
:103C60001AF0EACF1BF00001386B8FDC290E2EDC36
:103C70003A0E2CDC200E2ADC0001200E366F000EDE
:103C8000376F140EE8CF38F0F4DE0001200E366FE7
:103C9000000E376F00011C0E386F000E396F05DF04
:103CA000006E016A01500010D8A40AD000019B0EDA
:103CB000366F100E376FC3DE9EAAFED7AE501200CD
:103CC0001AC0E9FF1BC0EAFF1CC0EEFF1DC0EEFFDB
:103CD0001EC0EEFF1FC0EEFF12004A0EE96E020E7C
:103CE000EA6EEF50FE0B0109EF6E12004A0EE96E0C
:103CF000020EEA6EEF50FE0BEF6E1200E150310A39
:103D000001E158D7030A9BE0010A9DE0070A9FE002
:103D1000010AE3E0030AEAE0010AEFE00F0AEDE03E
:103D200012000001440E366F0F0E376F88DE17DF6A
:103D30000001196F390AD8B402D019511EDF0001F1
:103D40001951380AD8B41200ECD70F0E1DEF2DF020
:103D5000040E1DEF2DF0200ED96ED92EFED71200C5
:103D600043000001516B526B43C04FF044C050F010
:103D7000000147C0F6FF48C0F7FF010E4727000EBD
:103D80004823050EF76403D00800F55005D0F6CFA0
:103D9000E9FFF7CFEAFFEF504C6F00090001D8B4FC
:103DA000D1D2250AD8B40AD0514B522B46514511D5
:103DB000D8A484D14C5103EC00F0DAD700014A6951
:103DC0004B6B496B6CD2000146514511D8B406D0FB
:103DD00045C0E9FF46C0EAFF000EEF6A51C000F09F
:103DE00052C001F0120000015051016E4F51006E9F
:103DF000020E4F27D8B0502B00C0E9FF01C0EAFFE8
:103E0000EFCF4BF04CD20001498D49D20001492B34
:103E100006D0080E00014A27FE0E00014A270001C5
:103E20005051016E4F51006E020E4F27D8B0502BEB
:103E300000C0E9FF01C0EAFFEECF4DF0EDCF4EF03C
:103E400049A10ED04EAF07D04D1F4E1F4D2BD8B4F9
:103E50004E2B4B0707D00001499149AD03D0F9D74C
:103E6000000149910B0E00014A274A51026E036A74
:103E70004DC000F04EC001F0C1EC2CF000504C6F72
:103E80004A51026E036A4DC000F04EC001F0C1EC11
:103E90002CF004C04DF005C04EF0010E536F546B72
:103EA000000154514E5D02E153514D5DD8A010D038
:103EB00000014A51026E036A53C000F054C001F081
:103EC0006BEC2DF004C053F005C054F04B07E8D75D
:103ED00049A914D01AD00001514B522B465145111B
:103EE000D8B409D045C0E9FF46C0EAFF200EEF6E06
:103EF000454B462B03D0200E03EC00F000014B078E
:103F00004B51800A7F0FD8B0E6D749A114D00001E9
:103F1000514B522B46514511D8B409D045C0E9FF49
:103F200046C0EAFF2D0EEF6E454B462B16D02D0EE8
:103F300003EC00F012D049AD10D00001514B522BD0
:103F400046514511D8B406D045C0E9FF46C0EAFF46
:103F50002B0EE9D72B0E03EC00F049B914D04DD04D
:103F60000001514B522B46514511D8B409D045C0E0
:103F7000E9FF46C0EAFF300EEF6E454B462B03D0FB
:103F8000300E03EC00F000014B074B51800A7F0F0D
:103F9000D8A033D0E5D753C002F054C003F04DC0D1
:103FA00000F04EC001F0C1EC2CF004C000F005C0E0
:103FB00001F000014A51026E036AC1EC2CF000507E
:103FC0004B6F800A760FD8A002D0070E4B27000156
:103FD000514B522B46514511D8B40AD04B51300F9A
:103FE00045C0E9FF46C0EAFFEF6E454B462B05D0C2
:103FF00000014B51300F03EC00F000014A51026EFA
:10400000036A530EE96E000EEA6EEE50006EEF503A
:10401000016EC1EC2CF00550ED6E0450EF6EEE50C9
:10402000ED10D8A4B8D70A0E00014C5DD8A002D07C
:10403000070E4C270001514B522B46514511D8B465
:1040400008D04C51300F45C0E9FF46C0EAFFEF6E83
:104050003BD000014C51300F03EC00F089D6000139
:104060004B51800A7E0FD8A015D0514B522B465190
:104070004511D8B409D045C0E9FF46C0EAFF200E7B
:10408000EF6E454B462B03D0200E03EC00F00001F1
:104090004B07E5D75051016E4F51006E020E4F276E
:1040A000D8B0502B00C0E9FF01C0EAFFEFCF4CF0C1
:1040B000514B522B46514511D8B409D045C0E9FFA8
:1040C00046C0EAFF4CC0EFFF454B462B51D60001DE
:1040D0004C5103EC00F04CD600015051016E4F5191
:1040E000006E020E4F27D8B0502B00C0E9FF01C070
:1040F000EAFFEECF00F0EDCF01F000C012F001C0FA
:1041000013F0D96AD950006E016A12C0E8FF00248A
:10411000026E13C0E8FF0120036E02C0F6FF03C069
:10412000F7FF050EF76403D00800F55005D0F6CF71
:10413000E9FFF7CFEAFFEF500009D8B402D0D92A3F
:10414000E1D700014A51D95CD8B002D0D9504A6FAA
:1041500000014A514BBF42D0FF0A4B25D8A03FD0A7
:10416000514B522B46514511D8B409D045C0E9FFF7
:1041700046C0EAFF200EEF6E454B462B03D0200EC3
:1041800003EC00F000014B07E3D712C0F6FF13C0A9
:10419000F7FF050EF76403D00800F55005D0F6CF01
:1041A000E9FFF7CFEAFFEF5000014C6F0001122B3F
:1041B000000E13230001514B522B46514511D8B428
:1041C00009D045C0E9FF46C0EAFF4CC0EFFF454BB0
:1041D000462B04D000014C5103EC00F000014A07CB
:1041E0004A29D8B4C5D5D1D747C0F6FF48C0F7FF94
:1041F000050EF76403D00800F55005D0F6CFE9FFAF
:10420000F7CFEAFFEF502A0AD8A412D0000150518C
:10421000016E4F51006E020E4F27D8B0502B00C0D8
:10422000E9FF01C0EAFFEFCF4AF0474B482B37D0F8
:1042300047C0F6FF48C0F7FF050EF76403D008003B
:10424000F55005D0F6CFE9FFF7CFEAFFEF50D00FDA
:1042500000014A6F474B482B47C0F6FF48C0F7FFA5
:10426000050EF76403D00800F55005D0F6CFE9FF3E
:10427000F7CFEAFFEF50D96E300ED95CD8A00FD03F
:104280003A0ED95CD8B00BD04A510A0DD950F3245C
:10429000D00F4A6FCAD749B539D00001498900010A
:1042A00047C0F6FF48C0F7FF010E4727000E48231E
:1042B000050EF76403D00800F55005D0F6CFE9FFEE
:1042C000F7CFEAFFEF504C6F000A01E17CD52A0AD4
:1042D00001E189D5010A01E196D5050A85E01E0AAA
:1042E000DAE0680A01E195D53B0A01E1B8D6070A90
:1042F00001E18CD50B0A01E18FD51C0A01E1ECD656
:10430000060A01E18CD50D0A01E183D5300E0001CA
:104310004C5DD8A00CD03A0E4C5DD8B008D0498581
:104320004B510A0D4C51F324D00F4B6FB8D70001FD
:10433000514B522B46514511D8A4C0D64C5103ECD9
:1043400000F016D546514511D8B406D045C0E9FF56
:1043500046C0EAFF000EEF6A51C000F052C001F003
:1043600012009EBA9DAA09D1AB50060BD8B405D055
:10437000AB98AB88050EE8CF16F0AECF14F0180E50
:10438000E96E000EEA6EEF50FE0BEF6E160EE96E50
:10439000000EEA6EEF50010A23E0030A2FE0010A43
:1043A0003EE0070A70E0010A01E190D002C315F077
:1043B0000001176B14C0E8FFC00AD8A402D0030E96
:1043C00043D014C0E8FF410AD8A484D0180EE96E87
:1043D000000EEA6EEF50FE0B0109EF6E020E34D0B4
:1043E000180EE96E000EEA6EEF50FE0B0109EF6E3B
:1043F00014C0E8FF0D0AD8A46DD035D0180EE96EB0
:10440000000EEA6EEF50FE0B0109EF6E14C0E8FFDC
:10441000540AD8A402D0010E17D0050E15D0180EDC
:10442000E96E000EEA6EEF50FE0B0109EF6E14C04C
:10443000E8FFDB0AD8A40BD0180EE96E000EEA6E76
:10444000EF50FE0BEF6E040EE8CF16F043D014C011
:10445000E8FFC00AD8A43ED0170EE96E000EEA6E3F
:10446000EF50D8B409D0180EE96E000EEA6EEF5086
:10447000FD0B0209EF6E2ED0180EE96E000EEA6EEB
:10448000EF50FE0BF7D7180EE96E000EEA6EEF50F4
:10449000FE0B0109EF6E030EE8CF16F014C0E8FF23
:1044A000DC0AD8A402D0C00E06D014C0E8FFDD0A92
:1044B000D8A404D0DB0EE8CF14F00CD0180EE96EAF
:1044C000000EEA6EEF50FE0BEF6E02D015C002F345
:1044D0000001166B18C000F000A030D00301022BC1
:1044E000FA0E02C300F0005CD8B0026B00C300F00B
:1044F000020EE96E030EEA6EEF500018D8B413D026
:104500000001172B040E006E030E016E020EE96E01
:10451000030EEA6EEF500024E96E000E0120EA6EF1
:1045200014C0EFFF0BD015C002F30001166B180E7C
:10453000E96E000EEA6EEF50FD0BEF6E18C000F052
:1045400000A21BD0180EE96E000EEA6EEF50FD0BB4
:10455000EF6E040E006E030E016E150EE96E000E76
:10456000EA6EEF500024E96E000E0120EA6E02C3ED
:10457000EFFF0301012B0001166B9EA812009DA8FE
:104580001200000EE96E040EEA6EEF50D8B445D06A
:10459000040E006E016E010EE96E040EEA6EEF501D
:1045A0000024E96E000E0120EA6EEF50E8CF14F00F
:1045B00014C0E8FFC00AD8A412D0DB0EE8CF14F074
:1045C000040E006E016E010EE96E040EEA6EEF50ED
:1045D0000024E96E000E0120EA6EDC0E16D014C035
:1045E000E8FFDB0AD8A413D0DB0EE8CF14F0040EEA
:1045F000006E016E010EE96E040EEA6EEF500024AB
:10460000E96E000E0120EA6EDD0EEF6E03D00401AC
:104610000007012B14C0ADFF12009D9803C400F0E9
:1046200000A008D0030EE96E040EEA6EEF50FE0BF8
:10463000EF6E1200C00EAD6E1200000E1BD900010D
:10464000166B0001186B0301006B016B036B026BAF
:104650000501AF6B9E9A9D8A9D98200EAC6E900EC0
:10466000AB6E070EAF6EF28EF28C1200FA0E00C423
:1046700000F0005CD8A09DB8000C010C1F00010EDA
:10468000E8CFAFF5E96E030EEA6EEF50D8B4000C38
:1046900000C303F30301032BFA0E03C300F0005C15
:1046A000D8B0036B040E006E030E016EE96EEA6E65
:1046B000EF500024E96E000E0120EA6EEF50410A2F
:1046C000D8A41AD063D8030EE96E040EEA6EEF5038
:1046D000FE0B0109EF6E040EE8CF00F40401026B3B
:1046E0000501AF6B4F0E75D84B0E73D80D0E71D8F8
:1046F0000A0E6FD8B4D8000C21C0E9FF22C0EAFF2F
:10470000EF6A010CAFC5E8FF0009040E006ED8B4D3
:1047100014D0030E016E0301032B03050024E96E80
:10472000000E0120EA6EEFCFD9FFFA0E03C300F0AE
:10473000005CD8A00ED0036B0CD0040E016E0401F7
:10474000022B02050024E96E000E0120EA6EEFCF75
:10475000D9FFD9501200590000015C51016E5B5124
:10476000006E5B07D8A05C070110D8B40AD0CADF7E
:1047700059C0E9FF5AC0EAFFEF6E0001594B5A2BAE
:10478000EBD75BC000F05CC001F012009D9A010EF7
:10479000E96E030EEA6EEF50D8B411D0040E006E2D
:1047A000030E016EE96AEA6EEF500024E96E000E16
:1047B0000120EA6EEF50E8CF00F3030101079D8A64
:1047C0001200DA00DDC000F40401026B0501AF6BDA
:1047D0001200D96EAFC5E8FF0009040E006ED8B410
:1047E00014D0030E016E0301032B03050024E96EB0
:1047F000000E0120EA6ED9CFEFFFFA0E03C300F0DE
:10480000005CD8A01200036B1200040E016E0401BC
:10481000022B02050024E96E000E0120EA6ED9CFBA
:10482000EFFF1200DA00DAC0E1FFDBC0E2FF0001B7
:10483000DD51016EDC51006EDC07D8A0DD070110F0
:10484000D8B41200E250016EE150006EE14AE22A53
:1048500000C0E9FF01C0EAFFEF50BBDFE8D7040169
:10486000026B016B03C400F000B002D0C00EAD6E4D
:104870009D8812009DB812000401006B026B016B51
:10488000036B12008300E96A030EEA6EEF50000129
:104890008327000E8423834B842B845DF90ED8B4C8
:1048A000835DD8A005D08351060FE8CF03F302D073
:1048B00083C003F3010EE8CFAFF51200C100C1C001
:1048C00002F40501AF6B120012009D9A020EE96E10
:1048D000030EEA6EEFCFD9FF9D8A010EE96E030E3B
:1048E000EA6EEF50D8B41DD0D95000C300F0005C80
:1048F000D8B00FD0FA0E006E016AD950005E000EDB
:10490000015AE96A030EEA6EEF500026000E0122FA
:104910001200D95000C300F0016A005E000E015A77
:104920001200F80E006E016A12001F000001440E12
:10493000596F000E5A6F0001140E5B6F5C6BACEC8C
:1049400023F0F00E006E00014415400AD8A4B5D043
:1049500044C000F00F0E0016D8900036D8900034F6
:10496000EC0F276F150E275DD8B0A7D02751D8B40C
:104970000CD00001300E596F000E5A6F0001275104
:1049800000015B6F5C6BACEC23F04E0EE96E000E29
:10499000EA6EEECF2AF0EDCF2BF000014E6B4F6B9D
:1049A0000001440EDA6F000EDB6F0001140EDC6FA5
:1049B000DD6B8AEC26F0001C026E011C036E02C047
:1049C0002CF003C02DF000012751D8B415D0000100
:1049D000300EDA6F000EDB6F000127510001DC6F33
:1049E000DD6B8AEC26F0001C026E011C036E02C017
:1049F0002EF003C02FF003D000012E6B2F6B0001AF
:104A00002C0EDA6F000EDB6F0001040EDC6FDD6B25
:104A10008AEC26F000C028F001C029F00001440E05
:104A2000DA6F000EDB6FB9D8000129512B1902E1B2
:104A300028512A19D8A441D0F00E006E4415400A1E
:104A4000D8A43BD01FC0E1FF20C0E2FFE250E1103C
:104A5000D8B40CD0E1CFE9FFE2CFEAFF54C0EEFFBB
:104A600055C0EEFF56C0EEFF57C0EEFF0001060E28
:104A70002125E96E000E2221EA6E50C0EEFF51C0E2
:104A8000EEFF52C0EEFF53C0EEFF23C0E9FF24C08B
:104A9000EAFF4DC0EFFF2751465D006E4751D8A099
:104AA0004705016EEC0E002425C0E9FF26C0EAFF91
:104AB000EE6EFF0E0120ED6E010CC6EC23F0000C33
:104AC000C100450EE8CFC6F00001C76B140EC42527
:104AD000E8CFC8F0000EC521E8CFC9F00001102BC7
:104AE000000E112310C0CAF011C0CBF00001CC6B36
:104AF000CD6B640EE8CFCEF0C3C0CFF0D06BD16BDE
:104B000032C2D2F033C2D3F034C2D4F035C2D5F0C1
:104B1000060EC125E96E000EC221EA6EEECFD6F078
:104B2000EECFD7F0EECFD8F0EDCFD9F0ED52ED5279
:104B30000001C60EDA6F000EDB6F2FD80001C60E23
:104B4000DA6F000EDB6F0001140EDC6FDD6B8AEC98
:104B500026F000C0D0F001C0D1F0C1C0DAF0C2C070
:104B6000DBF00001DC6B0001140EC425E8CFDDF0A2
:104B7000000EC521E8CFDEF0E2EC23F00001C60E06
:104B8000DA6F000EDB6F0001140EDC6FDD6B13ECCF
:104B900024F0006A016A1200DA000001020EDA2530
:104BA000E96E000EDB21EA6EEECF00F0EDCF01F0F2
:104BB00000C0DCF001C0DDF021EC26F00001020EA7
:104BC000DA25E96E000EDB21EA6E00C0EEFF01C0BF
:104BD000EDFF040EDA25E96E000EDB21EA6EEECF62
:104BE00000F0EDCF01F000C0DCF001C0DDF021EC01
:104BF00026F00001040EDA25E96E000EDB21EA6ED4
:104C000000C0EEFF01C0EDFF0A0EDA25E96E000ECE
:104C1000DB21EA6EEECF00F0EDCF01F000C0DCF05A
:104C200001C0DDF021EC26F000010A0EDA25E96E64
:104C3000000EDB21EA6E00C0EEFF01C0EDFF1200A6
:104C4000DC0014D0DCC0DEF0DDC0DFF0DF0EE96E8A
:104C5000000EEA6EEFCFE0F0DEC0DFF0E0C0DEF085
:104C6000DEC000F0DFC001F000D01200EBD7C300BF
:104C70004FD0C3C0C8F0C4C0C9F0C5C0CAF0C6C0D8
:104C8000CBF00001C80ECC6F000ECD6F030ECC250B
:104C9000E96E000ECD21EA6EEFCFC7F0CCC0E9FF80
:104CA000CDC0EAFF030ECC25E16E000ECD21E26EF1
:104CB000EFCFE7FFCCC0E9FFCDC0EAFFC7C0EFFFF1
:104CC000020ECC25E96E000ECD21EA6EEFCFC7F0C3
:104CD000010ECC25E16E000ECD21E26E020ECC2538
:104CE000E96E000ECD21EA6EE7CFEFFF010ECC2575
:104CF000E96E000ECD21EA6EC7C0EFFFC8C000F01C
:104D0000C9C001F0CAC002F0CBC003F000D012004D
:104D1000B0D7DA0088D00001DE6BDF6BE06BE16BAF
:104D2000D890DD31E36FDC31E26FDAC0E4F0DBC054
:104D3000E5F01BD00001E551016EE451006E020E5A
:104D4000E427D8B0E52B00C0E9FF01C0EAFFEECFB1
:104D500000F0EDCF01F0026A036A0050DE27015037
:104D6000DF230250E0230350E1230001E351016EF1
:104D7000E251006EE207D8A0E30701500010D8A46A
:104D800001D001D0D7D7DCA101D001D00ED0E4C032
:104D9000E9FFE5C0EAFFEF500001DE27010ED8B0C1
:104DA000DF27D8B0E027D8B0E1272BD00001E651AB
:104DB000046EE751056E066A076AFF0EDE15006E87
:104DC000FF0EDF15016E000EE015026E000EE115FC
:104DD000036E04C0E8FF0024086E05C0E8FF012050
:104DE000096E06C0E8FF02200A6E07C0E8FF032034
:104DF0000B6E08C0DEF009C0DFF00AC0E0F00BC0A7
:104E0000E1F0E0C0E6F0E1C0E7F00001E751E611B3
:104E1000D8A401D001D0CAD70001DE1D006EDF1D6D
:104E2000016E00D0120077D793002ED093C096F079
:104E300094C097F017D0610E0001955DD8A007D0FF
:104E400000D07B0E955DD8B002D000D002D000D04B
:104E500006D096C0E9FF97C0EAFFE00EEF260001FA
:104E6000964B972B96C0E9FF97C0EAFFEF500001E1
:104E7000956F0009D8A401D001D0DDD793C000F010
:104E800094C001F000D01200D1D793002FD095C06C
:104E90009AF096C09BF093C098F094C099F019D006
:104EA0009AC0F6FF9BC0F7FF98C0E9FF99C0EAFFE0
:104EB000050EF76403D00800F55005D0F6CFE1FFEA
:104EC000F7CFE2FFE750EF6E0001984B992B9A4B1A
:104ED0009B2B000197079729D8A401D001D0E0D7D8
:104EE00093C000F094C001F000D01200D0D71F0092
:104EF0000001310E596F000E5A6F0001080E5B6FF2
:104F00005C6BACEC23F0330EE96E000EEA6EEECF74
:104F10002BF0EDCF2CF00001336B346B0001310E20
:104F2000DA6F000EDB6F0001080EDC6FDD6B8AECC0
:104F300026F0001C026E011C036E02C02DF003C09F
:104F40002EF023C0E1FF24C0E2FFF80EE72621C0C7
:104F500059F022C05AF0E75000015B6F5C6BACEC7B
:104F600023F021C0DAF022C0DBF023C0E9FF24C027
:104F7000EAFFEF500001DC6FDD6B8AEC26F0001CCD
:104F8000026E011C036E02C02FF003C030F000015E
:104F90002D0EDA6F000EDB6F0001040EDC6FDD6B8F
:104FA0008AEC26F000C029F001C02AF00001310E81
:104FB000596F000E5A6F86D81FC0E9FF20C0EAFF64
:104FC00031C0EFFF25C0E9FF26C0EAFF35C0EEFF84
:104FD00036C0EDFF27C0E9FF28C0EAFF37C0EEFF6B
:104FE00038C0EDFF00012C512A1902E12B5129197B
:104FF000000ED8B4010E12001F0000012A6B21C060
:1050000029F02B6B2C6B25C02DF026C02EF027C06D
:105010002FF028C030F00001310E5F6F000E606F7E
:1050200022C061F023C062F0000124510001636FCF
:10503000646B8AEC2CF00001290E596F000E5A6F38
:1050400041D80001290EDA6F000EDB6F00012451F8
:10505000006E016A080E0024E8CFDCF0000E01208B
:10506000E8CFDDF08AEC26F000C02BF001C02CF078
:105070001FC0C1F020C0C2F0010EE8CFC3F0000194
:105080002451006E016A080E0024E8CFC4F0000E1F
:105090000120E8CFC5F061EC25F00001290EDA6FA0
:1050A000000EDB6F00012451006E016A080E00241F
:1050B000E8CFDCF0000E0120E8CFDDF013EC24F0A7
:1050C0002FEF24F00001040E5925E96E000E5A213D
:1050D000EA6EEECF00F0EDCF01F000C0DCF001C0D1
:1050E000DDF021EC26F00001040E5925E96E000EDA
:1050F0005A21EA6E00C0EEFF01C0EDFF060E5925F1
:10510000E96E000E5A21EA6EEECF00F0EDCF01F00D
:1051100000C0DCF001C0DDF021EC26F00001060E3D
:105120005925E96E000E5A21EA6E00C0EEFF01C05B
:10513000EDFF020E5925E96E000E5A21EA6EEECF00
:1051400000F0EDCF01F000C0DCF001C0DDF021EC9B
:1051500026F00001020E5925E96E000E5A21EA6E72
:1051600000C0EEFF01C0EDFF120007D00501AE6BDD
:105170000501AD6B010E00D01200F8D77F009ED064
:10518000ADC500F000A001D001D003D0006A016AD3
:1051900094D00001B30E906F0E0E916F7FC0E9FFA7
:1051A00080C0EAFFEF50D8A401D001D005D0FF0E97
:1051B000006EFF0E016E81D07FC093F080C094F02E
:1051C00015EC27F000C07FF001C080F070D0000126
:1051D000810E936F000E946F90C095F091C096F081
:1051E0000F0EE8CF97F046EC27F0810EE96E000E27
:1051F000EA6EEF50D8A401D001D038D07FC093F030
:1052000080C094F0F5EC2CF000500001926F0D0E70
:10521000925DD8A001D001D002D00C0E926F7FC059
:1052200093F080C094F00001840E956F000E966F8D
:10523000000192510001976F986BCAEC2BF001505E
:105240000010D8A401D001D00BD00501AE2B820EE6
:10525000E96E000EEA6EEECF00F0EDCF01F02DD03A
:105260000F0E00019027000E912321D081C0E8FF8E
:10527000040AD8A401D001D015D000018351FF0A3F
:10528000FF0ED8B48219D8B401D001D009D0820E53
:10529000E96E000EEA6EEECF90F0EDCF91F001D006
:1052A00007D005D0FF0E006EFF0E016E06D08FD71F
:1052B000FF0E006EFF0E016E00D0120061D713D0FA
:1052C0000501AC6BAD0EE96E050EEA6EEF50FE0BFC
:1052D000EF6EAEC5E8FF0009D8B401D001D002D00E
:1052E0000501AE071200ECD741D0FEC1F6FFFFC1A9
:1052F000F7FF050EF76403D00800F55005D0F6CF90
:10530000E9FFF7CFEAFFEF500001836F0101FE2BA9
:10531000000EFF2300018351030AD8A401D001D05D
:1053200015D0FEC1F6FFFFC1F7FF050EF76403D0ED
:105330000800F55005D0F6CFE9FFF7CFEAFFEF50B0
:10534000836F0101FE2B000EFF230CD0000183515F
:10535000040AD8A401D001D005D0FF0EE8CFFEF199
:10536000E8CFFFF10001835100D01200BED70DD06D
:10537000AD0EE96E050EEA6EEF50FE0B0109EF6E01
:10538000200E006E016A00D01200F2D705D0000195
:10539000196F010E00D01200FAD706D0FEC100F03E
:1053A000FFC101F000D01200F9D70501B06B1DEC70
:1053B00023F0B1EC02F0EEEF08F00001196B192BAD
:1053C00000011951D8B4A0EF0CF0196BD2D0000134
:1053D000510E1F6F020E206F00011A0E216F000E7A
:1053E000226F3FEC23F0006E016A015000100001B3
:1053F000D8B4E7D7196B192B1A51D8A402D0020ED2
:105400003CD000011A51060AD8A402D0050E35D0AE
:10541000C6EC23F0D5D70001196BB6EC02F00009F9
:10542000D8B4CED731D000011B0E1F6F000E206FF5
:105430000001510E216F020E226F00011A0E236F20
:10544000000E246F00014B0E256F020E266F96ECA6
:1054500024F0006E016A01500010D8B418D0000189
:10546000196B192B1A05D8A402D0030E06D000011F
:105470001A51060AD8A404D0060EE8CFB0F5A0D77A
:105480000001196BC6EC23F00501B06B99D7C6EC8F
:1054900023F0FAD70001510E1F6F020E206F4BC28E
:1054A00021F04CC222F0A2EC0CF0006E016A015017
:1054B0000010D8B402D00501B06B0001196B80D781
:1054C0000501B06B0201000E4C5D2A0ED8B44B5D95
:1054D000D8B02ED000011A0E1F6F000E206F0001F1
:1054E000B10E216F050E226F00014B0E236F020ECD
:1054F000246F00014D0E256F020E266F00014F0E26
:10550000276F020E286F78EC27F0006E016A0150B9
:105510000010D8B40BD000011A51080AD8A406D044
:10552000196B192B040EE8CFB0F502D00501B06B52
:10553000C6EC23F045D736EC23F00009D8B440D7A9
:105540000001510E1F6F020E206F0001216B000140
:10555000B10E226F050E236F4BC224F04DC225F011
:105560004EC226F04FC227F050C228F0FDEC27F0C3
:105570008BD7B0C5E8FF000A01E129D7010A01E194
:1055800026D7030A01E14FD7010A9AE0070AD3E0C0
:10559000010A01E140D7030A01E17CD7E0EF29F0DD
:1055A00037D0F00E83160F0E9512959A9598929A11
:1055B000839A8398809AA5EC1EF0F00E9516F00E53
:1055C00083168382808A00F000F0809AA8EC1EF097
:1055D000F00E83168382808A00F000F0809AABEC94
:1055E0001EF0F00E83168382808A00F000F0809A0D
:1055F0000F0E9512280E0DD8080E0BD80C0E09D8D8
:10560000010E07D8130E05D8800E03D800D0120063
:10561000C8D72CD00001436F00D029D80009D8A4E6
:1056200001D001D0FAD7959A9598F00E9516F00E04
:105630008316000143390F0B8312839A839800F07D
:1056400000F0808A00F000F0809AF00E83160F0EB2
:10565000006E00504315831200F000F0808A00F0C5
:1056600000F0809A0F0E951200D01200D3D723D0ED
:10567000959A9598838A839800F000F0808A00F0CC
:1056800000F083A601D001D00BD0809A00F000F08A
:10569000808A00F000F0809A839A010E0BD00AD025
:1056A000809A00F000F0808A00F000F0809A839ADF
:1056B000000E00D01200DCD7430014D006D0000149
:1056C000455132D80001434B442B43C0E9FF44C04D
:1056D000EAFFEF500001456F0009D8A401D001D0C6
:1056E000EED71200EBD743001ED006D00001455183
:1056F0001BD80001434B442B43C0F6FF44C0F7FFC7
:10570000050EF76403D00800F55005D0F6CFE9FF89
:10571000F7CFEAFFEF500001456F0009D8A401D090
:1057200001D0E4D71200E1D733D00001466F00D09A
:105730009EDF0009D8A401D001D0FAD7959A959898
:10574000F00E9516F00E83160F0E006E46C001F097
:10575000013A0F0E01160050011483128388839AB8
:1057600000F000F0808A00F000F0809AF00E8316BE
:105770000F0E006E000100504615831200F000F07D
:10578000808A00F000F0809A0F0E951200D012006F
:10579000CCD7930000019851016E9751006E970786
:1057A000D8A098070110D8B45ED093C0F6FF94C07B
:1057B000F7FF050EF76403D00800F55005D0F6CFCB
:1057C000E9FFF7CFEAFFEF500009D8B422D095C027
:1057D000F6FF96C0F7FF050EF76403D00800F550FA
:1057E00005D0F6CFE9FFF7CFEAFFEF50006E93C088
:1057F000F6FF94C0F7FF050EF76403D00800F550DC
:1058000005D0F6CFE9FFF7CFEAFFEF500018D8B484
:1058100024D093C0F6FF94C0F7FF050EF76403D0C1
:105820000800F55005D0F6CFE9FFF7CFEAFFEF50BB
:10583000006E016A95C0F6FF96C0F7FF050EF7648B
:1058400003D00800F55005D0F6CFE9FFF7CFEAFF07
:10585000EF50005E000E015A12000001934B942B92
:10586000954B962B97D7006A016A12008F008FC064
:1058700002F090C003F091C0F3FF92C0F4FF00016A
:105880009451016E9351006E9307D8A094070110B4
:10589000D8B43CD0F3CFF6FFF4CFF7FF010EF326D8
:1058A000000EF422050EF76403D00800F55005D071
:1058B000F6CFE9FFF7CFEAFFEF50016E02C0F6FF27
:1058C00003C0F7FF010E0226000E0322050EF76447
:1058D00003D00800F55005D0F6CFE9FFF7CFEAFF77
:1058E000EF50006E0150005C0001956F966BD8A0E0
:1058F000960700BE960701BE962B96519511D8B417
:10590000BED795C000F096C001F01200006A016A8F
:1059100012005F0061C0F3FF62C0F4FF5FC0D9FFF7
:1059200060C0DAFF00016451016E6351006E6307CD
:10593000D8A064070110D8B41FD0F3CFF6FFF4CF7E
:10594000F7FF010EF326000EF422DA50016ED95053
:10595000006ED94ADA2A00C0E9FF01C0EAFF050E4D
:10596000F76403D00800F55005D0F6CFE1FFF7CF7C
:10597000E2FFE750EF6ED6D75FC000F060C001F0E5
:105980001200066A046A056A0250031003E1006A05
:10599000016A000C1F0E0612D890062A0236033642
:1059A000FCE3033202320250005C0350015804E36E
:1059B000016E0250005ED88004360536062E06BA07
:1059C000F0D706AE05D0041E042AD8B40506051E7D
:1059D0000450026E0550036E06AC000C001E002A37
:1059E000D8B40106011E000C930093C0F3FF94C0CD
:1059F000F4FFF3CFF6FFF4CFF7FF010EF326000E0E
:105A0000F422050EF76403D00800F55005D0F6CF58
:105A1000E9FFF7CFEAFFEF500009D8A4EAD7000169
:105A20009351F35C006E9451F458016EFF0E002404
:105A3000006EFF0E0120016E120022D000011A6FCD
:105A400017D00001040E196F0CD00001500E1B6F0F
:105A500003D000011B6B1B2B01D000D000011B2FBA
:105A6000FCD7000119071929D8A401D001D0EDD71E
:105A700000011A071A29D8A401D001D0E2D71200D8
:105A8000DDD75E0ED66EF80ED76E070ED56ED58EAC
:105A9000F284F28A12005BC200F05CC201F01200D4
:105AA000F2A41200F80ED76E5E0ED66E02015B2BCA
:105AB000000E5C238978F2941200EFCF00F0EE2AFA
:105AC000EFCF01F0000EEE22EFCF02F0EE22EFCF8B
:105AD00003F0EE22120002500002F3CF04F0F4CFE4
:105AE00005F00102F350052603500002F35005268D
:105AF0001200D96E3A0ED95CD8B006D0300ED95CFF
:105B0000D8A002D0D8801200D89012000900F5CF9A
:105B1000EEFFEA50E262FAD7E950E162F7D71200ED
:0A5B2000EECFE6FFE82EFCD7000CE4
:020000040030CA
:04000000FFFAFCFE09
:020000040000FA
:00000001FF
